:100000000C308A005D2C0000503472346534763434
:1000100072346134633465346E34FD3420347034AA
:1000200061346E3465346C3429340D340A34003450
:1000300050346F3464346134F83465346E34E934E8
:1000400020346E34613473347434613476346534FE
:100050006E34ED343A34203425344C3464340D3469
:100060000A340034C135E332EC32F237ED32743900
:100070003A10A0060A00533A613B202C3A1025267C
:1000800064147039EF316537F430A9060A00533A29
:10009000613BA02C3A10252664147039EF31653786
:1000A000F430A9060A00533A613B202D3A10252668
:1000B00064147039EF316537F430A9060A007A34D8
:1000C0006134643461346E34FD3420347534683402
:1000D00065346C3420342534643420340D340A34CF
:1000E000003483168611831286110830F8007828B0
:1000F0000000F8178928F813C90C03188615031C8B
:100100008611781789287813F80B7C288728000037
:1001100086153F308400840B8B280000F81B7B2859
:10012000781B83280800831603178C170C14000013
:10013000000083120C087F390319D7280313B60077
:1001400003170D080313B70003170F080313B800B4
:100150003608C9007120370803178D0003133808CB
:1001600003178F0083168C170C14000000008312F5
:100170000C0D0E0D7F390319D7280313B600031792
:100180000D080313B70003170F080313B800360850
:10019000C9007120370803178D00031338080317AF
:1001A0008F008D0A03198F0A031393280317031373
:1001B0008A150A12D12C3F08013A0319E328033AA1
:1001C0000319EC28F52883168810831288108316EB
:1001D000081083120814FD288316081083120810D3
:1001E0008316881083128814FD28831688108312C2
:1001F0008810831608108312081008000830F800D1
:10020000000086108316861000008312CD0D0610A4
:10021000031C0D2983160614831203181229831652
:1002200006108312831686148312861C1529F80B78
:1002300000290000861083168610000006140000B6
:10024000000086148312861C2329F801000006187A
:1002500078148610831686108312061083160610F3
:10026000831208008316061400008614000083120F
:10027000061083160610000083128610831686105F
:1002800038308312CD00FE202A30CD00FE20013010
:10029000CD00FE2083160610000086148312861CF3
:1002A0004F29000053290000831606140000831212
:1002B0008A150A12DB2C0830CE007708CF0083168F
:1002C0000614000086148312861C64290618031481
:1002D000061C0310F80D000083168610831286108A
:1002E000CE0B5F29831606140000831206104F08F8
:1002F00003197D29831606108312000083168614C5
:100300008312861C81290000861083168610000047
:10031000831206108316061083120800C901CA0151
:10032000831606140000861400008312061083163C
:100330000610000083128610831686103830831250
:10034000CD00FE204708CD00FE20831606140000D5
:10035000861400008312861CAB2906108316061033
:100360000000831286108316861039308312CD0068
:10037000FE20F7015B217808CA00831606100000F2
:1003800086148312861CC2290000C6290000831629
:1003900006140000061400008614000083120610E4
:1003A00083160610000083128610831686103830DC
:1003B0008312CD00FE204808CD00FE2083160614CF
:1003C0000000861400008312861CE42906108316A0
:1003D00006100000831286108316861039308312AF
:1003E000CD00FE20F7015B217808C90083160610B6
:1003F000000086148312861CFB290000FF290000E0
:100400008316061400008312CE014A08CD00CE00E8
:10041000CD0149084D07F8004E08FA000318FA0A02
:100420007808CB007A08CC004C08CE004B08CD00F1
:10043000D0010430CF004E0850068039D200CE1FC4
:10044000262ACD09CE09CD0A0319CE0AD01F2D2A9E
:10045000CF09D009CF0A0319D00AF801F901F70131
:10046000FA015008031D372A4F080319512A10308A
:10047000D1000310CD0DCE0DF70DFA0D50087A0204
:10048000031D442A4F087702031C4D2A4F08F70228
:10049000031CFA035008FA020314F80DF90DD10BEE
:1004A000392AD21F582AF809F909F80A0319F90A52
:1004B0007908CC007808CB004B08F8004C08F9000C
:1004C0000800831603178C170C1400000000031893
:1004D000902A83120C087F390313B70003170D0805
:1004E0000313B80003170F080313B9003708C90036
:1004F0007120380803178D000313390803178F0084
:1005000083168C170C140000000083120313B60B23
:100510008A2A8D2A83160317902AAF2A8316031777
:1005200083120C0D0E0D7F390313B70003170D084E
:100530000313B80003170F080313B9003708C900E5
:100540007120380803178D000313390803178F0033
:100550008D0A03198F0A03100313B60B612A0800D2
:10056000C7010408C6004710831B4714C01FC02AD8
:10057000C617461EC60ABF09C009BF0A0319C00A2A
:10058000400EF038C200C207E23EC300323EC50052
:1005900040080F39C307C307C507E93EC400C407B5
:1005A000C4073F0E0F39C407C507C40DC50DC509E3
:1005B000C50D3F080F39C507C20D0730C1000A300D
:1005C000C507C403031CE02AC407C303031CE42AB1
:1005D000C307C203031CE82AC207C103031CEC2A99
:1005E00041308400831307304605461384034605D3
:1005F000031D012B461A840A461A012B2030F700EE
:100600001E2B840745300402031946170008F70023
:10061000031D122B461B122B461A2C2BC619122B0C
:1006200020301D2BC61F1A2B2D30F70084034613D4
:10063000C6131E2BC61546123030F707C00104083A
:10064000BF004010831B40147708C90071203F0889
:100650008400831340188317840A461F022B080066
:100660003F308400831300080319432B0230F80045
:10067000F701F70B392BF80B382B9730F700F70BF6
:100680003F2B800B362B08008E30F7004C08F8000B
:100690004B08F900FA01CC1F522BF809F909F90AA5
:1006A0000319F80AF808031D5F2B7908F800F9010F
:1006B0000830F702F808031D5F2BF701682B0310C1
:1006C000F81B662BF90DF80DF7035F2BCC1FF81301
:1006D00008005C0803192E2CE800600803192E2C72
:1006E000E802031C782B7F30E80703182E2C7E2BA2
:1006F0008130E802031C2E2C03192E2C6808F70009
:10070000F801F901FA01E7015D08E600E6175E0865
:10071000E5005F08E4001930E8006308E40203180C
:10072000A12B0130E5020318A12BE6020318A12B2F
:10073000E7020318A12BE70AE60AE50A6308E407C3
:10074000D32B6208E5020318BC2B0130E602031824
:10075000BC2BE7020318BC2BE70AE60A6208E50790
:100760006308E407031CD32BE50A031DD32BE60A19
:10077000031DD32BE70AD32B61088038E602031848
:10078000D22B0130E7020318D22BE70A6108803828
:10079000E6076208E507031CB02BE60A031DB02B31
:1007A000E70AB02B7A14E80BD62BE12B0310E40DEB
:1007B000E50DE60DE70D0310FA0DF90DF80DE90D45
:1007C0008D2B691CE92B0310F80CF90CFA0CE90CC1
:1007D000EC2BF70303192E2CE91B152C0310E40D49
:1007E000E50DE60DE70D6308E4020318012C013066
:1007F000E5020318012CE6020318012CE702031C92
:10080000242C6208E50203180C2C0130E6020318C0
:100810000C2CE702031C242C61088038E602031824
:10082000152C0130E702031C242CFA0A031D242C8A
:10083000F90A031D242CF80A031D242CF70A0319B6
:100840002E2CF80CF90CFA0C5D08E8006108E8069B
:10085000E81F2C2CF817322CF813322CF701F80172
:10086000F901FA0108005908E0005D08E006E01F00
:100870003E2C03110310D91B0314712C5908E000FE
:100880005C08E1005808E10203194C2CE01F712CB0
:100890000308013A8300712C5D08E1005908E10268
:1008A0000319582CE01F712C0308013A8300712CA6
:1008B0005E08E1005A08E1020319642CE01F712C64
:1008C0000308013A8300712C5F08E1005B08E10234
:1008D0000319702CE01F712C0308013A8300712C5E
:1008E000031008005C080319E22CE40060080319F7
:1008F000E22CE4070318832C7F30E402031CE22C73
:100900000319E22C872C8130E4070318E22C6408D9
:10091000F700F801F901FA015D08E800E8175E0840
:10092000E7005F08E6001830E400E501661CB02C23
:100930006308FA07031CA22CF90A031DA22CF80A6B
:100940000319E5176208F907031CA92CF80A031913
:10095000E5176108DE00DE175E08F8070318E517E3
:10096000E50DF80CF90CFA0CE80CE70CE60C03109A
:10097000E40B952C0130F7070318E22CF81BC72C69
:10098000E80DFA0DF90DF80DF7030319E22CE81F35
:10099000D82CFA0A031DD82CF90A031DD82CF80A02
:1009A000031DD82CF80CF90CFA0CF70A0319E22CE9
:1009B0005D08E5006108E506E51FE02CF817E62C68
:1009C000F813E62CF701F801F901FA01080080306C
:1009D0008318E106E601E7015D08E5006108E50628
:1009E0005C080319D72DE400F70060080319E02D17
:1009F000E40203197C2D031C3A2D6108EA00EA1772
:100A00006208E9006308E800E7010310EA0CE90C5A
:100A1000E80CE70CE40B042DE51F112D6614F42DF2
:100A20006610641066165F3084008313092E661208
:100A3000E51B242D641C2F2DEA0CE90CE80CE70CB7
:100A4000F70A0319EF2D2F2DEA1B322D0310E70DA6
:100A5000E80DE90DEA0DF7030319EF2D242D6617B4
:100A60009C2D66135D08E500E51F382DEA17E82D7B
:100A7000EA13E82D6008E400F7005C08E4025D0872
:100A8000EA00EA175E08E9005F08E800E7010310E2
:100A9000EA0CE90CE80CE70CE40B462DE51F532D9E
:100AA000E614F42DE6106410E61663308400831318
:100AB000092EE612E51B662D641C712DEA0CE90C6B
:100AC000E80CE70CF70A0319EF2D712DEA1B742DC2
:100AD0000310E70DE80DE90DEA0DF7030319EF2DFB
:100AE000662DE6179C2DE6136108E500E51F7A2DBB
:100AF000EA17E82DEA13E82D6108EA00EA17620810
:100B0000E9006308E800E51F892DEA136615F42D56
:100B10006611E70164105F3084008313092EE51B22
:100B2000B22D5D08E500641C9C2DEA0CE90CE80C74
:100B3000E70CF70A0319EF2DE71FAD2DE80A031D97
:100B4000AD2DE90A031DAD2DEA0A031DAD2DEA0CFA
:100B5000E90CE80CF70A0319EF2D661B312DE61B93
:100B6000732DD12D8030EA06EA1FBA2DF42D6108CD
:100B7000E500C72D5D08E500EA08031DC72DE9085B
:100B8000031DC72DE808031DC72DF701E82DEA1B3B
:100B9000D12D0310E70DE80DE90DEA0DF70BC72D78
:100BA000EF2DE51FD52DEA17E82DEA13E82D600893
:100BB000F7006108EA006208E9006308E800E82D30
:100BC0005C08F7005D08EA005E08E9005F08E800DD
:100BD0006A08F8006908F9006808FA00272EF7018A
:100BE000F801F901FA01272EE701E809E909EA0904
:100BF000E709E70A031D022EE80A031D022EE90A8F
:100C00000319EA0A6618102DE618522D6619882D68
:100C1000B72D0008E807031C132EE90A031D132E45
:100C2000EA0A0319641484030008E907031C1B2E55
:100C3000EA0A0319641484030008801F803AEA0753
:100C400003186414661A172DE61A592D8F2D080003
:100C50008E30F7003F08F7024008F9004108F8001D
:100C6000F917F70803193F2E0310F908031D3B2E4F
:100C7000F80803193F2EF90CF80CF70B342EC01F9F
:100C8000462EF809F909F80A0319F90A080083162B
:100C900003178C170C140000000083120D080313B7
:100CA000C00003170F080313C10003170C08031338
:100CB000C9007120400803178D0003134108031772
:100CC0008F008D0A03198F0A0313BF0B472E0800EC
:100CD0008A1500208A117A08BA007908B9007808C4
:100CE000B8007708B7003A08C2003908C1003808D0
:100CF000C0003708BF0028267908BC007808BB0070
:100D00003C08003C03188E2EFF3A031D8B2E3B0837
:100D10005E3C03188E2EBC01BB018E2E3B083602B2
:100D2000BF00C0013C08031C3C0FC0024008BE00CD
:100D30003F08BD00BE08031DA12E3D08023C03185C
:100D4000F32E3B083602031DA82EBC080319F22E11
:100D5000BC08031DB32E36083B020318B32E023025
:100D6000BF00DB20B62E0130BF00DB203230BF00D9
:100D700030230330BF00DB203230BF0030238A1520
:100D800000208A117A08BA007908B9007808B800FA
:100D90007708B7003A08C2003908C1003808C00017
:100DA0003708BF0028267908BC007808BB003C083B
:100DB000003C0318E52EFF3A031DE22E3B085E3C83
:100DC0000318E52EBC01BB01E52E3B083602BF002F
:100DD000C0013C08031C3C0FC0024008BE003F0895
:100DE000BD00A12E9A2E0330BF00DB201830031760
:100DF0008D0000308F0014300313BF0047261030E1
:100E000084003C08C0003B08BF00B0220D30C90080
:100E100071200A30C90071208A150A12772D3D0809
:100E2000F8013C020318172F3C08F700232FF701A5
:100E30000830BE00BC0DF70D3D0877020318F7001F
:100E4000F80DBE0B1A2F08002030371E3030B800C6
:100E50003608F700B61F332FF709F70A7708B600F0
:100E60002D30B800B7173608BC006430BD000F271E
:100E70007708B60030307807B9003608BC000A3071
:100E8000BD000F2730307707BB0030307807BA003D
:100E90003808F700B71D4E2FB71F3711371A5B2FD1
:100EA000B71F762F3719762F7708B900B718762F26
:100EB0007708BA00762F30303902031D762F770875
:100EC000B9002030B800B71D692F3711B714B71F0C
:100ED000B71030303A02031D762F7708BA00203061
:100EE000B900B71D692FB710B71F3710371D7B2FFB
:100EF0003808C9007120B71C802F3908C90071203B
:100F0000371C852F3A08C90071203B08C9007120A1
:060F10008A150A12892D6A
:101000000130C7000230C8008A118E218A15790884
:10101000A1007808A0000330C7000430C8008A117E
:101020008E218A157908A3007808A2000530C70030
:101030000630C8008A118E218A157908A500780823
:10104000A4002108FA002008A11F2F282008003C36
:10105000F700FA012108031C210FFA027708A60005
:101060007A08A7002308FA002208A31F40282208B4
:10107000003CF700FA012308031C230FFA0277084B
:10108000C7007A08C800FA304707A8004808A90036
:101090000318A90A2508FA002408A51F58282408BF
:1010A000003CF700FA012508031C250FFA02770817
:1010B000C7007A08C800FA304707AA004808AB0002
:1010C0000318AB0A2308CC002208CB008A11442362
:1010D0008A157708C7007808C8007908C9007A0817
:1010E000CA002508CC002408CB008A1144238A15A5
:1010F0004A08DF004908DE004808DD004708DC0038
:101100007A08E3007908E2007808E1007708E00057
:101110008A1169238A157A08C2007908C100780803
:10112000C0007708BF004208CA004108C900400853
:10113000C8003F08C7005710D7104A08CE0049081A
:10114000CD004808CC004708CB004A08DB0049081E
:10115000DA004808D9004708D800DF01DE01DD01C8
:10116000DC018A1133248A15031CBA2857144C0851
:10117000803ACC00DB01DA01D9017F30D8004E087B
:10118000DF004D08DE004C08DD004B08DC008A1152
:1011900033248A15031CE528DF01DE01DD017F30E1
:1011A000DC004E08E3004D08E2004C08E1004B086B
:1011B000E0008A1169238A157A08CE007908CD00EB
:1011C0007808CC007708CB00D7140A30DF008930CC
:1011D000DE003430DD007C30DC004E08E3004D08DA
:1011E000E2004C08E1004B08E0008A1172248A15E5
:1011F0007708D8007808D9007908DA007A08DB0087
:10120000DF007908DE007808DD007708DC004E0892
:10121000E3004D08E2004C08E1004B08E0008A11B1
:1012200072248A157708D8007808D9007908DA007E
:101230007A08DB0083107A08DF007908DE0078087E
:10124000DD007708DC007C30E3007930E2003530E7
:10125000E1008130E0008A11E7248A157A08D20083
:101260007908D1007808D0007708CF005208DF0055
:101270005108DE005008DD004F08DC004E08E30096
:101280004D08E2004C08E1004B08E0008A1172248E
:101290008A157708D8007808D9007908DA007A0822
:1012A000DB00DF007908DE007808DD007708DC006D
:1012B0004E08E3004D08E2004C08E1004B08E00056
:1012C0008A1172248A157708D8007808D90079081D
:1012D000DA007A08DB0083107A08DF007908DE0084
:1012E0007808DD007708DC003F30E3000230E200E0
:1012F0003330E1008330E0008A11E7248A157A0850
:10130000D2007908D1007808D0007708CF005208C1
:10131000DF005108DE005008DD004F08DC004E08F9
:10132000E3004D08E2004C08E1004B08E0008A11A0
:1013300072248A157708D8007808D9007908DA006D
:101340007A08DB00DF007908DE007808DD00770826
:10135000DC004E08E3004D08E2004C08E1004B08B9
:10136000E0008A1172248A157708D8007808D9001D
:101370007908DA007A08DB0083107A08DF00790840
:10138000DE007808DD007708DC003330E3008C30C5
:10139000E2001E30E1008330E0008A11E7248A1564
:1013A0007A08D2007908D1007808D0007708CF00F9
:1013B000DF01DE01DD017F30DC004E08E3004D0877
:1013C000E2004C08E1004B08E0008A1172248A1503
:1013D0007708D8007808D9007908DA007A08DB00A5
:1013E000DF007908DE007808DD007708DC004E08B1
:1013F000E3004D08E2004C08E1004B08E0008A11D0
:1014000072248A157708D8007808D9007908DA009C
:101410007A08DB0083107A08DF007908DE0078089C
:10142000DD007708DC001B30E300E430E2003530FB
:10143000E1008230E0008A11E7248A157A08D6009C
:101440007908D5007808D4007708D3005608DF0063
:101450005508DE005408DD005308DC004E08E300A8
:101460004D08E2004C08E1004B08E0008A117224AC
:101470008A157708D8007808D9007908DA007A0840
:10148000DB00DF007908DE007808DD007708DC008B
:101490004E08E3004D08E2004C08E1004B08E00074
:1014A0008A1172248A157708D8007808D90079083B
:1014B000DA007A08DB0083107A08DF007908DE00A2
:1014C0007808DD007708DC00A430E300DB30E200C0
:1014D0006730E1008330E0008A11E7248A157A083A
:1014E000D6007908D5007808D4007708D3005608CC
:1014F000DF005508DE005408DD005308DC004E080C
:10150000E3004D08E2004C08E1004B08E0008A11BE
:1015100072248A157708D8007808D9007908DA008B
:101520007A08DB00DF007908DE007808DD00770844
:10153000DC004E08E3004D08E2004C08E1004B08D7
:10154000E0008A1172248A157708D8007808D9003B
:101550007908DA007A08DB0083107A08DF0079085E
:10156000DE007808DD007708DC003330E3008C30E3
:10157000E2001E30E1008330E0008A11E7248A1582
:101580007A08D6007908D5007808D4007708D30007
:101590004E08DF004D08DE004C08DD004B08DC0083
:1015A0005208E3005108E2005008E1004F08E00053
:1015B0008A1172248A157708D8007808D90079082A
:1015C000DA007A08DB00DF007908DE007808DD0049
:1015D0007708DC005608E3005508E2005408E100F3
:1015E0005308E0008A1169238A157A08D200790825
:1015F000D1007808D0007708CF00D71C1B2B8314AC
:10160000DB30DF000F30DE004930DD007F30DC00F2
:101610005208E3005108E2005008E1004F08E000E2
:101620008A11E7248A157A08D2007908D10078084F
:10163000D0007708CF00571C202B5008803AD000EC
:101640004F08F7005008F8005108F9005208FA0056
:101650007A08C6007908C5007808C4007708C30076
:101660004608DF004508DE004408DD004308DC00D2
:10167000C330E300F530E2004830E1008030E000A4
:101680008A1169238A157708C7007808C800790885
:10169000C9007A08CA00DF004908DE004808DD00FA
:1016A0004708DC00E301E2013430E1008630E0006D
:1016B0008A1172248A157A08C6007908C50078084C
:1016C000C4007708C3004308F7004408F800450841
:1016D000F9004608FA00F8134608C6004508C50098
:1016E0007808C4004308C300A91F792BA71F962BB5
:1016F0007B2BA71B852B29082702031C852B031D89
:10170000962B26082802031C962BAB1F8A2BA71F9B
:10171000962B8C2BA71BBF2B2B082702031CBF2B40
:10172000031D962B26082A020318BF2B043003172B
:101730008D0000308F0083168C170C140000000001
:1017400083128C080319BD2B0D080313C700031760
:101750000F080313C80003170C080313C9008A11EC
:1017600071208A15470803178D00031348080317D3
:101770008F008D0A03198F0A9B2B532C0313A40887
:10178000031DDA2BA508031DDA2BA31BD52BA308F9
:10179000031DCE2B2208003C0318D52BC601C50122
:1017A0003430C4008630C300D92BC601C501C40142
:1017B000C301522CA51B1B2CA508031DE32B2408D9
:1017C000003C03181B2CA31B002C8310DF01DE013F
:1017D0003430DD008530DC004608E3004508E200D7
:1017E0004408E1004308E0008A11E7248A157A08DA
:1017F000C6007908C5007808C4007708C3001A2C11
:101800008314DF01DE013430DD008530DC00460862
:10181000E3004508E2004408E1004308E0008A11C3
:10182000E7248A157A08C6007908C5007808C4003C
:101830007708C300522CA31B382C8314DF01DE0170
:101840003430DD008630DC004608E3004508E20065
:101850004408E1004308E0008A11E7248A157A0869
:10186000C6007908C5007808C4007708C300522C68
:101870008310DF01DE010730DD008730DC00460821
:10188000E3004508E2004408E1004308E0008A1153
:10189000E7248A157A08C6007908C5007808C400CC
:1018A0007708C300031703134308F7004408F80040
:1018B0004508F9004608FA000800840183131F3028
:1018C0008305713083168F000F08861183128615E9
:1018D000831603170908C039890003131F129F12CA
:1018E0000030031788008312870188018901FF30C7
:1018F0000313AC00831603170908C03989000313CA
:101900001F129F12003003178800831203131F1346
:101910009F1383169F1383121F149412AC122C086A
:101920008316870083122C162C08831687008312D7
:10193000AC112C088316870001308312940000300C
:10194000831694000108C73908388100831290017A
:101950000030F800920000308316920083122C159C
:101960002C08831687008312970183169B019C0124
:1019700001309D00831203178701880189018316B6
:101980000908C039890003131F129F12283003175A
:101990008800323083128D0000308F008A110313CB
:1019A00093288A150330BF008A11DB208A150A307C
:1019B000B5008A1132298A150130C7000230C800EB
:1019C0008A118E218A157908A1007808A0000330B9
:1019D000C7000430C8008A118E218A157908A30037
:1019E0007808A2000530C7000630C8008A118E2191
:1019F0008A157908A5007808A4003B3003178D00EC
:101A000000308F00031008300313B6008A116122E2
:101A10008A15103084002108C0002008BF008A11F8
:101A2000B0228A15403003178D0000308F00031458
:101A30000C300313B6008A1161228A154730031750
:101A40008D0000308F00031008300313B6008A1198
:101A500061228A15103084002308C0002208BF00CC
:101A60008A11B0228A154C3003178D0000308F0088
:101A700003140C300313B6008A1161228A15533007
:101A800003178D0000308F00031008300313B600D9
:101A90008A1161228A15103084002508C0002408AC
:101AA000BF008A11B0228A15583003178D0000300C
:101AB0008F0003140C300313B6008A1161228A15BB
:101AC0000030F8001F08C33978049F009F140130CC
:101AD000BF008A1130238A159F186C2D9F149F1800
:101AE0006F2D1E08B5003508B6008A11682E8A15BC
:101AF0005F3003178D0000308F000C300313BF00E0
:101B00008A1147268A153508B6001F30B7008A119A
:101B1000242F8A152030C9008A1171208A150D30B2
:101B2000C9008A1171208A150A30C9008A117120F2
:101B30008A150830B600FA30BF008A1130238A15A2
:081B4000B60B9B2DDC2C6300A9
:04400E00F52CFF3F4F
:00000001FF
